:10000000830100308A0091288C0003088301B4002A
:100010002D08B5002E08B60083122008023C810787
:100020000B119D0B6D289D0A6628051A6D2803107B
:100030001F0CAD002D032228051A252803101F0CC4
:10004000AD002D0A9D009E0A6D289E016D281108A5
:10005000AD00AE010230AD070318AE0A1E082D0632
:100060002E0403195D280830990A190203183C2848
:10007000051E53289B0A5328990104301B029B013B
:1000800003189B0A1B08AD001103AE00AE0A4A28F4
:100090000310AD0DAE0B48282D08AD0003101C0C4D
:1000A0002D049C009E0A1F08AD000310AD0C031028
:1000B000AD0C03102D0C9D006D281C089A000D1628
:1000C0009D019D0A9C019E0199016D281E0803193E
:1000D0001528013A03191C28272813080319712829
:1000E0009303FF30A507031CA60326082504031D60
:1000F0007E282308A5002408A6000D150D1C8728BE
:100100008F030F0A03198728083085068F00831292
:100110003508AD003608AE00340883008C0E0C0E96
:1001200009000D3084000E309E200E3084002D30EA
:100130009E208301302A04068001840A04060319E4
:1001400000349B28820745340A3441342034533428
:10015000493455340D34443452344A344E344634E0
:1001600043344B3454345A344C345734483459346F
:10017000503451344F344234473400344D345834C1
:100180005634820733340A342D342034273438343B
:1001900037340D3423343434F4342C3440343A348A
:1001A000283435342B342934323424343634303442
:1001B000313439343F342A3400342E342F343D3432
:1001C00082078034803480344034403420348207C5
:1001D000AB349C3468349C348E34683482071734D2
:1001E0001A341D3420342334263482072B342E3421
:0201F0003134A8
:1001FA008312AB00861559298312A800FD203229E3
:10020A008312AB008611592901308312052103306C
:10021A001C2983120D1E0F290D121A0808008312B9
:10022A00AB00890083160814831208080800831299
:10023A00A900120893001308031D2029A90B1E29DF
:10024A0008008312AA002E29AA0A2A031421FD20D3
:10025A008312A903290F292908008312900A3C292D
:10026A00403090003A29C2211008803E0529100822
:10027A00183A03193529403A031D08003829B101F3
:10028A00B2010310B00CAF0C031C52292D08B107A0
:10029A002E0803182E0AB2070310AD0DAE0D2F0853
:1002AA0030040319003446298312AC000F30860546
:1002BA002C08F0398604061506110F3086052C0E17
:1002CA00F039860406150611013093001308031944
:1002DA0008006B298312AA008316881872298312D0
:1002EA002A0889002908880003108B1B03148B1322
:1002FA008316081555308900AA3089008814081118
:10030A0003188B17831208008312AA014030A90030
:10031A000330A700A02907308605290886040A3079
:10032A00A800A80B96290518A229AA0A8518A229A5
:10033A00AA0A0310A90DA70B90292A080800F03071
:10034A008316860083128614861506150608AC00E5
:10035A000611F030AC0506150608AB0006112B0E87
:10036A000F39AC048316860183128610013093007C
:10037A001308031DBD292C0808008312AA01D629D7
:10038A002A08C03E83120521A421A9002A08C03EDA
:10039A0005212030FD202A08803E05212908FD205C
:1003AA00AA0A18302A02031CC529C0308312052163
:1003BA00403090000800831209219001063005217F
:1003CA001730A90000302621C03005210230A900CB
:1003DA00293026210330A90000308A000E08EE20B9
:1003EA0026210330A900343026210330A900003029
:0603FA008A001708F5203F
:1004000026210530A9003730262121084E3EFD283F
:100410001330831685008601831206149D019D0A00
:100420009E018D129C010D12990105158511083050
:100430008F008D11A20198012308A5002408A600B1
:100440000D110A3094000230960004309500831696
:10045000811283122008023C81008B168B17080042
:100460003C30831214218E003D30142197003E3021
:100470001421A100822208225822E0210D14051126
:10048000FA301C210D10FA301C2105150D1A8D199A
:10049000512A8D1A4E2A8D168312092183120E219C
:1004A000B4220D1D462A0D11831289212F23462ABD
:1004B0008312861086111E301C210F3086053030C5
:1004C00086040615061105301C210615061101309B
:1004D00093001308031D692A0615061105301C2117
:1004E0000F30860586160615061101309300130895
:1004F000031D772A28300521083005210C300521FD
:100500000630052900308A0083120E08E0209F0083
:1005100000308A000E08E720A0009708031D922AE9
:1005200005309100170B962A073091001708023A00
:10053000031D9C2A083091002008AF00B001E8306C
:10054000AD000330AE00B1233108AD002D0A92009A
:100550003230AF00B0011208AD00AE0144213108C5
:10056000A3003208A40008008312A70005150D108F
:100570009708031DE52A1F30A705A70803190800DF
:1005800027081B3A031DC62A8D14080027081F3AA6
:10059000031DCC2A8D1008002708043A031DD72A12
:1005A000210BD32A8D102108023A03198D14A703B9
:1005B0008D1CE02A00308A002708C120A7000D2BDF
:1005C00000308A002708A220DE2A80302702031C80
:1005D0000D2BA030270203180D2B0730A7050D2B7C
:1005E00027085A3A031DF82A18080A3A0319022B59
:1005F000A2012708433A0319022BA20127085A3AFD
:10060000031D042BA20A192BA2012708433A031D3C
:10061000192BA20105110D14192B22080319F02A18
:10062000013A0319F92A033A0319FE2A013A031978
:10063000052B27080D3A031D252B1808270603193B
:10064000252B051127089800C22920302702031CFA
:100650000800270883120121270898000800831248
:10066000A700043A031D3C2B1508043A031D3A2B3E
:10067000A801A12B0230492B1508043A031D452B74
:10068000A801A80A27089500A12B940803194B2B51
:100690000330A800A12B0430492B0A3094009601A6
:1006A000960A08008030831205218D157D2B0630B7
:1006B0008E0A0E02031C892B8E01892B0330970AA8
:1006C0001702031C892B9701892B0330A10A2102F1
:1006D000031C892BA101892B05110E08A9003C30B0
:1006E0006F211708A9003D306F212108A9003E3075
:1006F0006F21051509218D11892B27080319572B07
:10070000013A03196C2B033A03195E2B013A0319C2
:10071000652B2703031908008222E0290A30940080
:100720009601960A0430950008009408031D94036E
:100730000800960B0800023096000800043095006F
:100740000800280803194D2B013A0319522B033ACC
:1007500003198E2B013A0319952B073A0319992B8C
:100760009E2BB301AE1FBB2BAD09AD0A0319AE031F
:10077000AE093317B31730088039B306B01FC72B43
:10078000AF09AF0A0319B003B009C72BB301B10118
:10079000B2012F083004031DD02BAD01AE0100348F
:1007A0001F30B3040310B30AAF0DB00D031CD32BDD
:1007B000B00CAF0C30082E02031DE02B2F082D02C9
:1007C000031CE82B2F08AD023008031C300AAE02D0
:1007D000B10DB20DB30BB31AD82BB31FF42BB10963
:1007E000B10A0319B203B2093108AF003208B000F0
:1007F000331F0034AD09AD0A0319AE03AE0900344E
:02400E00F13F80
:10420000540054005900200031002E0034002000DA
:1042100042002E00560045004C004C004500200096
:104220002800430029003200300030003300340001
:104230003500200035003000200037003500200018
:1042400031003000300031003100300033003000E8
:10425000300053003A0054004C0058004100530015
:10426000370041005300380020004D003A00200084
:1042700055004F0053003A0002000000000000000B
:00000001FF
